:100000000200AF000000000000000000000000003F
:1000100000000000000000000000000209200000B5
:100020000000000D0A0D0A4D432D322039393034BD
:1000300031392D322E303076202020200D0A4D45CA
:1000400054434F4E2D32203939303431392D322E30
:10005000303076202020436F707972696768742091
:10006000286329205061756C204E65776C616E6441
:100070002C20502E452E2020313939322D3139395E
:10008000392E2020416C6C205269676874732052AD
:10009000657365727665640D0A002020202020209B
:1000A000202020202020202020202020202000C2CE
:1000B000AF75D00078FF7600D8FCC2AF75D0007560
:1000C00081AF1209D31209E91209F6120FD0120BEF
:1000D00044C200C20112012792001202339201822F
:1000E000004003120245120E46D2AF120F0F20003D
:1000F000031210D02001031210F9020DB7C0A8C2DC
:10010000AF3127D0A8300F030210D0513340061270
:1001100002450210F922512EC0A8C2AF314BD0A81F
:10012000A20F12176901FD7CA47D107E117824C2F4
:100130000DC20ED20C31B0200F0DC20C0C318D202F
:100140000D05200E02D322D20FC32278247CA47D79
:10015000107A11315F50040DDAF9D3D20FC322C2E5
:100160000DC20ED20C7CA47E01319D200D06200E06
:1001700003D32177C3D20FC0D03181D0D022000069
:10018000221201847E367F00DFFEDEFA2231B520A6
:100190000E0631D7F608DEFA510BD20F2231B52008
:1001A0000E09E60831F2200EEFDEF7510BD20F22D6
:1001B00031B5510B22D20BC20DC20E3096143097BE
:1001C000115126511CEC31F2200E06300C03ED319A
:1001D000F222D20DD20F227F085114A29733511C64
:1001E000DFF7BE0104512121EB51265114511C515E
:1001F00021227F08339297512B5114511CDFF55166
:10020000215114309702D20E511C22512651145103
:1002100021C20B22D2963096FD512B22C296512B31
:1002200022D297512B22C297512B22000022513308
:10023000EBF72279347B10E427240319DBFAFB6700
:10024000C37001D32279257B10900254E493F709FF
:10025000A3DBF92205000012345641000000000023
:10026000000000000012102640030210AF12105FC1
:10027000121065EFFA742C2EF8E60A13DAFD9200DC
:10028000121012EF2430120A21742D120A21A2003A
:10029000120F9A120F1C2212102640030210AF12E6
:1002A000105FEFFA742C2EF8D30AE433DAFD46F629
:1002B00080BE12102640030210AF12105FEFFA74D6
:1002C0002C2EF8D30AE433DAFDF456F680A212108D
:1002D0002640030210AF8FF012105FEFFA742C2E3D
:1002E000F8D30AE433DAFD20F005F456F6808146AF
:1002F000F6417012102640030210AF742C2EF8E65F
:10030000FC121065121012742D120A21EC1203C295
:10031000120FB0EC120F69120FB0EC120F86120F11
:100320001C2212102640030210AF742C2EF8EFF698
:1003300080C9121026400302005F12036812106584
:10034000121012742D120A2112037C120FB0ED123A
:100350000F69EC120F69120FB0ED120F86120FB376
:10036000EC120F86120F1C22742C2EF8E6FC08E605
:10037000FD18E66C70F208E66D70ED2279007A00E7
:100380007B00ECFEEDFF7006EE700302039F12038C
:10039000AC1EEE7004EF6007EEB4FFF21F80EFEBCF
:1003A000120F75EA120F69E9120F6922E92401D4CC
:1003B000F9400122EA2401D4FA400122EB2401D4BD
:1003C000FB2275F064842430120A21E5F075F00AEE
:1003D000842430120A21E5F02430120A2122E61882
:1003E000120F86120FB0DEF6221210659014A112C1
:1003F0000F29782F7E0471DE9014F4120F299015C6
:100400000B120F2978347E0571DE901546120F29E4
:10041000901560120F2978397E0571DE90159B12B8
:100420000F29783E7E0571DE9015B5120F29758370
:1004300021758208AE837168717C15831583120F54
:10044000B3D582F0901672120F2975833175820828
:10045000AE837168717C15831583120FB3D582F05A
:10046000901691120F29121065120FB39016B21246
:100470000F29221205DF120B791414147911B4001C
:100480000A12106512061A120F1C22B40644120634
:10049000047A00B40400400A2496D4CA2404D4CABE
:1004A00080F1C0E0EA7880F6D0E0C4232354C0FA9B
:1004B0007875E6543F4AF6120604541FFA08E654CB
:1004C000E04AF6120604543FFA18E654C04AF6020F
:1004D000054EB40415120604543FFA7874E654C06D
:1004E0004AF612060418F602054EB4020E1206046D
:1004F0007872F6E418F618F602054EB40135E7B442
:100500002B127872E6B45905760002054E2401D408
:10051000F602054EB42D127873E6B4000576590242
:10052000054E2499D4F602054EB430077872760051
:1005300002054EB430004020B43A00501B140303AF
:100540000354E0FA7876E6541F4AF602054E120587
:10055000F412106512061A2202108E1205DF120B19
:100560007914790FB40007120672120F1C22B40618
:100570001F120604120604541FFA787EE654E04A5D
:10058000F6120604543FFA18E654C04AF60205D59E
:10059000B40415120604543FFA787CE654C04AF6B7
:1005A00012060418F60205D5B4020C120604787A75
:1005B000F6E418F60205D5B4050F1206047870F6B5
:1005C0001206047878F60205D5B4031012060478F2
:1005D0007EF60205D51205F41206722202108E7CF8
:1005E000A07D007E13787075F000D20C31B0C20C83
:1005F0000C318D227CA07D007E13787075F000D2C6
:100600000C319D22E709120FD1C4FAE709120FD16C
:100610004A22E709120FD1540F22B1DF7875E6C4E0
:1006200003035403C0E07880E6FAD0E02AD4120F26
:10063000697876E6541F120F6918E6543F120F6965
:10064000742F120A2118E6543F120F6918E6120F90
:1006500069742F120A2118E6120F69742F120A21E9
:100660009006DF7876E6C4035407FA1206D3120F19
:100670002922B1DF7458120A21120A21787EE65429
:100680001F120F6918E6543F120F69742F120A21C6
:1006900018E6543F120F6918E6120F69742F120AF8
:1006A0002118E6120F69742F120A21120A2178709C
:1006B000E6120F697878E6120F697478120A2174CD
:1006C0002F120A21787EE6120F697478120A21121D
:1006D0000F1C22EA700122E493A370FBDAF9225383
:1006E000554E004D4F4E005455450057454400545B
:1006F0004855004652490053415400FF120AE94050
:100700000122780EE6643D600122E52B08E6652BA8
:10071000600122200506200603020B8608E608B4C5
:1007200053024197B4430241B2B444024165B4520A
:100730000302078CB457030207A0B4480690116C5B
:10074000020F29B44D0261E9B454028173B4560317
:10075000020F0FB45A10753A00753B00753C0075D6
:100760003D00753E0022B445030207AFB4580302B2
:10077000114FB44C03020B8CB44603020807B4417A
:1007800002A15BB44F030208CD02108EE608B4420A
:10079000024165B4590241F3B45702613202108E2E
:1007A000E608B4420241CEB45902612202108EE63C
:1007B00008B4570B512EC2AF314BD2AF0207C2B4AF
:1007C000521BC0A8C2AF3127D0A851336005514594
:1007D0000210F99007EF121065120F2922B4440C91
:1007E00020060302111E51451210782202108E209D
:1007F000454550524F4D2057524954452F5245417F
:1008000044204F4B0D0A00E608B45557E65407B490
:100810000007782C7A3102083EB40107782C7A0957
:1008200002083EB4020778357A0A02083EB403078C
:10083000783F7A1002083EB40426784F7A101210DE
:10084000657428120A217B00E6120F69E6042BFB6F
:1008500008DAF5EB120F697429120A21120F1C2213
:1008600002108EB444FA782C7C00120A1412100B79
:10087000120FD1503CFA120A1412100B120FD15061
:10088000306A702D120A1412100B120FD15022FB75
:10089000120A1412100B120FD150166B7013EAC407
:1008A0004BFBE824D4FE1210455006EBF6080C80F2
:1008B000B9120F1C1210659008C5120F29EC120F07
:1008C00069120F1C224C4F414445442D002006055F
:1008D00012111EC322E608B44212E65407FAE525B7
:1008E00054F84AF5259016F4120F2922B44D2EE63D
:1008F0005407B40009C22CC22DC22E020916B4013D
:1009000009D22CD22DD22E020916B40210D22CC23A
:100910002DC22E0209169016F4120F292202108EF3
:10092000C0D0C0E0C082C08375D008051AE51AB4F3
:10093000243C751A00D207E51C6007200204D2028D
:10094000151CE51B2401D4F51B500D751B00120965
:1009500077051CD203020962540FB400053062020D
:10096000D203E51BA2E192B520E0031209ABD083CC
:10097000D082D0E0D0D032A81E08E52D13D8FD409B
:100980000FE51E25E0243FF8C28EA68B08E58DF604
:10099000051EE51EB40803751E0074F85290E51E8E
:1009A0004290758B00758D00D28E2290F8FDE0FB91
:1009B000656C8B6C5B552DFB783F7A08EB13FB5015
:1009C0000DE62401F608E63400F6080209D008080E
:1009D000DAEA22740044024450F589758C00D28C06
:1009E000D28E75B80275A8022290F8FF748AF09032
:1009F000F8FC74FFF02275985043878075C83475F1
:100A0000CBFE75CAE0D29922120A8CA29822120A51
:100A10008CA29922120A8C3098FAC298E599547FD8
:100A200022120A8C20060320140E3099F4B40A0412
:100A3000302E0122C299F5992230030EC203120A08
:100A40004B120A5D120A68120A7C2290F8FDE0300F
:100A50003001F4F535FF655F423A8F5F2290F8FC74
:100A6000E530203101F4F022E522540F90F8FEF039
:100A7000E054F0FAE522540F4AF52222E5353030F1
:100A800001F454807003C20622D20622100701220C
:100A9000A293B3929322C294120AB91392950000C2
:100AA000D2940000C294DFF37F09D2940000C29474
:100AB000A2B433DFF5120AC422C0E090F8FF740636
:100AC000F0D0E022C0E090F8FF7407F0D0E02212EE
:100AD0000F1CA214121769E5355480121755A2068F
:100AE000121769A2051217692251084001225114F8
:100AF000120B4C7002C322AA0CA80DB4081CE50C02
:100B0000B40002C322740812100B742012100B746C
:100B10000812100B150C150DC322B40D11A80D767B
:100B200000740D12100B740A12100B020B441210F9
:100B30000B120B68F608050C050D7600E50C24F584
:100B400050D680D9750C00750D0ED322B47F037476
:100B50000822B40903742022B40D0122B408012232
:100B6000FF24E0EF4001E422FF249FEF4001222414
:100B700085EF500122EF24E022790E7F00E7600428
:100B80000F0980F9EF2208E6B44C3B08E6B44304B1
:100B9000120C5222E6B4410A20060302111E120C66
:100BA0008B22B44F4FC205756A00756B0012106539
:100BB000900BB7120F29224C4F47474544204F5501
:100BC000540D0A00056B121065900BD3120F2912F9
:100BD0000C5222212121204552524F522C20555394
:100BE0004552204D555354204C4F47494E2021210A
:100BF000210D0A00B449CF087928E764FF602C1260
:100C00001026E76E70BE09E76F70B912102609E76B
:100C10006E70B1D205121065900C1F120F29224C74
:100C20004F4747454420494E0D0A0009E7F583091F
:100C3000E7F58279677A03121017E709120D0C6F36
:100C40007082DAF380CD7A037867120C76F608DAD0
:100C5000F9229146121065900C6F120F297A0378D1
:100C600067E608120F69120FB3DAF6120F1C22435F
:100C700048414C3A20007964E72411F7FB09E72446
:100C800025F76BFB09E72443F76B22120F19900C31
:100C9000FE120F297A037828E6120F6908DAF99014
:100CA0000D05120F297A107B00EB120F69120FB39A
:100CB0000BDAF6120F1C120FAA7A10742D51215163
:100CC00021120FB3DAF5120F1CE529F583E52AF599
:100CD000827A007B107C00EA120F69743A5121126B
:100CE0000FB3EA2410FA7D10EC120D0C0C120F69F0
:100CF000120FB3DDF3120F1CDBDD120F1C22534564
:100D000045443A20000D0A2020202000641C9365F1
:100D10008365822425648322302C03301407756A8E
:100D200000756B002220050CE56A24C44007E56BC2
:100D300024FC400122121065900D73120F29740AD1
:100D4000120DA5900D97120F297403120DA5900D89
:100D50009B120F297405120DA5C2B1D21074051291
:100D60000DA5D2B1C210900D9F120F29756A0075A2
:100D70006B00222121212054494D4544204F5554D8
:100D8000202D20444953434F4E4E454354494E472E
:100D9000202121210D0A00030303000D440D000D45
:100DA0002020200D00F404F5F0756A00C0F0D0F0AA
:100DB000E56A25F050F6221206FC120E2FB11851EA
:100DC00039120DD1120DF3120E46120E9B518C806A
:100DD000E630041EC204202B0330051612106512E3
:100DE000061A9016CC120F2920630122782C7A2B38
:100DF000114122202B03300535783A79357A05E602
:100E00005527600A7B087CFF130C4007DBFA0809B2
:100E1000DAED22C313DBFDF6E9C3942CFE12106554
:100E200012061A9016DE120F29ECFF1202732230FE
:100E30001405C205020E45300605D205020E45E531
:100E4000287002D20522E5255407B4000775CBF3BC
:100E500075CABB22B4010775CBFB75CA8022B402E8
:100E60000775CBFE75CAE022B4030775CBFF75CAC0
:100E70007022B4040775CBFF75CAB822B405077594
:100E8000CBFF75CADC22B4060775CBFF75CAEE220C
:100E9000B4070775CBFF75CAF72222051FE51FB4FB
:100EA0000803751F00E51FC313FAE52FCA6006CAC1
:100EB0001A030380F7CA540320E022E51F251F24EC
:100EC0004FF8E51FA2E19200A2E292E1A20092E2B5
:100ED000D333D3337F055196F608760022A2E192F0
:100EE00001E51F251F244FF8E51FC313A2E0920060
:100EF000A2E192E0A20092E1A20133C333D3337F97
:100F0000055196F608760008F6087600051F22902F
:100F10000023120F29120F3322120F1CC0E0740D90
:100F20005121740A5121D0E022E493700122512111
:100F3000A380F69000007C007D00E4932CFC50011F
:100F40000DA3E583B417F3E582B4A6EE90115FF12B
:100F500029ED120F69EC120F69F11CF11C22E583D7
:100F6000120F69E582120F6922C0E0C4120F75D01A
:100F7000E0120F7522540F24F620D705243A020FF1
:100F80008324415121227F0433120F9ADFFA120F7A
:100F9000B37F0433120F9ADFFA22C0E040057430A9
:100FA000020FA574315121D0E022120FB3120FB3FA
:100FB000120FB3C0E074205121D0E022C0E0C0F095
:100FC000E0F5F0A3E0F582E5F0F583D0F0D0E02283
:100FD00022F5F024D05030E5F024C64006E5F05468
:100FE0000FD322E5F024BF501EE5F024B94006E5FA
:100FF000F024C9D322E5F0249F500CE5F024994059
:1010000006E5F024A9D3227400C322202D03120A7E
:101010002122EE120F6922E6120FD1C4FF08E61258
:101020000FD14FFF0822E6120FD1C4FE08E6120FBF
:10103000D14EFE08E6120FD1C4FF08E6120FD14FC1
:10104000FF08021045EE20E70624CD4010D32230E1
:101050000608F40424F850F5C32212111EC322EF2F
:10106000C4540FFF22742D120A21E52B120A217499
:101070002D120A21120FB3221165901081120F292F
:1010800022434F4D4D414E44204F4B0D0A001165F8
:10109000901097120F29223F3F3F20434F4D4D4163
:1010A0004E44204552524F52203F3F3F0D0A0011FF
:1010B000659010B8120F29223F3F3F20414444520F
:1010C000455353204552524F52203F3F3F0D0A0097
:1010D00011659010D9120F29223F3F3F20454550FE
:1010E000524F4D205452414E534645522045525284
:1010F0004F52203F3F3F0D0A001165901102120F21
:1011000029223F3F3F20454550524F4D20444154F6
:1011100041204552524F52203F3F3F0D0A0011657A
:10112000901127120F29223F3F3F204F4E4C59204C
:10113000464F522053595354454D2041444D494E3A
:101140004953545241544F52203F3F3F0D0A0078BB
:101150007FE670031880FAE8120F69120F1C224311
:101160006865636B73756D3A203078000D0A4249EB
:1011700054205245414420414E4420575249544541
:1011800020434F4D4D414E44530D0A3D7352426131
:10119000616220202020524541442053544E207348
:1011A0002C20414444524553532073732C20424910
:1011B0005420620D0A3D7357426161626420202011
:1011C0002057524954452053544E20732C204144FB
:1011D00044524553532073732C20424954206220BB
:1011E0004441544120640D0A0D0A4259544520528D
:1011F00045414420414E4420575249544520434FD5
:101200004D4D414E44530D0A3D73525961612020AA
:10121000202020524541442053544E20732C20411D
:101220004444524553532073730D0A3D735759611B
:1012300061646420202057524954452053544E2065
:10124000732C20414444524553532073732C204443
:1012500041544120425954452064640D0A0D0A57F7
:101260004F5244205245414420434F4D4D414E443E
:101270000D0A3D73525761612020202020524541C4
:101280004420574F5244204F462053544E20732C35
:1012900020414444524553532073730D0A0D0A3DB7
:1012A000734D454D4F525920202053484F572043EE
:1012B000555252454E54204D454D4F5259204449A8
:1012C00053504C41590D0A3D735645522020202061
:1012D000202053484F572043555252454E542056D4
:1012E000455253494F4E20414E44205349474E4F9B
:1012F0004E204D4553534147450D0A3D735A4150C9
:101300002020202020205A415020414C4C2043488E
:10131000414E474520494E50555453204241434B7E
:1013200020544F205A45524F0D0A3D7345524541B6
:10133000442020202052454144204441544120462D
:10134000524F4D20454550524F4D0D0A3D73455764
:101350005249544520202057524954452044415475
:101360004120544F20454550524F4D0D0A3D734585
:1013700044454620202020204745542044454641EE
:10138000554C5420454550524F4D20444154410D39
:101390000A0D0A41444452455353455320414E449B
:1013A0002042495420504F534954494F4E532041F5
:1013B000524520414C5741595320494E20484558E9
:1013C00020283136292E20204F555450555420497D
:1013D0005320414C574159530D0A42415345203146
:1013E0003020464F4C4C4F574544204259204241F3
:1013F000534520313620464F4C4C4F5745442042F0
:1014000059204241534520322E0D0A0D0A3D735496
:101410006E6E6E6E6E6E20205345542054494D45BD
:101420002079796D6D64642C2068686D6D2C207353
:10143000732C20444F573D20312D372C2061646A96
:101440002F6D6D3D202B202D2C2061646A2F73732E
:101450003D20300D0A3D73416E6E6E6E6E6E202023
:1014600053455420414C41524D2079796D6D64644F
:101470002C2068686D6D2C2073732C20444F573DD1
:1014800020312D372C2061646A2F6D6D3D202B207B
:101490002D2C2061646A2F73733D20300D0A0D0AD4
:1014A0000053544154555320444953504C41590D15
:1014B0000A0D0A2020202020202020202020414426
:1014C000432D54595045202020204144432D43466C
:1014D0004720202050554C312F4643545220202085
:1014E0002053544154300D0A202020202020202059
:1014F0002020200053595354454D202830332030AC
:1015000032203031203030290D0A000D0A202054BD
:10151000582D533320202020202054582D53322082
:10152000202020202054582D5331202020202020FE
:1015300054582D5330202020202054582D50342F23
:101540004120200D0A005458202020202028303827
:10155000203037203036203035203034290D0A0035
:101560000D0A202052582D533320202020202052B5
:10157000582D533220202020202052582D53312026
:10158000202020202052582D53302020202020526F
:10159000582D50352F4220200D0A0052582020206F
:1015A0002020283044203043203042203041203059
:1015B00039290D0A0052582D43484720283132203E
:1015C0003131203130203046203045290D0A2D2D73
:1015D0002D2D202D2D2D2D20202D2D2D2D202D2D6F
:1015E0002D2D20202D2D2D2D202D2D2D2D20202D6C
:1015F0002D2D2D202D2D2D2D20202D2D2D2D202D4F
:101600002D2D2D20200D0A37363534203332313040
:1016100020203736353420333231302020373635EC
:1016200034203332313020203736353420333231D4
:1016300030202037363534203332313020200D0A27
:101640000D0A202037202020202036202020202096
:10165000352020202020342020202020332020204E
:101660002020322020202020312020202020300D5A
:101670000A00462F5020435452532028483A4C2009
:101680002032323A32312D2D31343A3133290D0A9C
:101690000041444320524547532028483A4C2020DB
:1016A00033323A33312D2D32343A3233290D0A0D8B
:1016B0000A004D454D4F525920444953504C415911
:1016C00020434F4D504C4554450D0A004155544F51
:1016D0002054494D454F5554200D0A0D0A00494EDE
:1016E00050555420535441545553204348414E477C
:1016F000453A20004F4B0D0A00C0E0743B120A210E
:10170000D0E0C0E0120F69120FB3E8120F69120F98
:10171000B3E9120F69120FB3EA120F69120FB3EB9C
:10172000120F69120FB3EC120F69120FB3ED120F03
:1017300069120FB3EE120F69120FB3EF120F691295
:101740000FB3E5F0120F69120FB3743B120A2112A6
:101750000F1CD0E022C0E0743B120A21D0E0C0E0B0
:10176000120F69120FB3D0E022C0E0C0D0743B1258
:101770000A21D0D0C0D0E433120F75120FB3D0D0ED
:10178000D0E022C0E0743B120A21E5D0120F6912AA
:101790000FB3D0E022C0E0742D120A21E8120F69C5
:0717A000120FB3D0E022009C
:00000001FF
